:100000008A110A120528000009008B0183160E30A0
:100010009F00831283168501831283168601831243
:100020008316870183128316810183128B130B13AE
:10003000061186118316061186110F30860583126C
:10004000C830A0000030A1006F203330CB20333007
:10005000CB203330CB202230CB202830CB200F30A8
:10006000CB200130CB200130CB20E830A000033082
:10007000A1006F200130CB206230B4206F30B4205B
:100080006E30B4206A30B4206F30B4207530B420A4
:100090007230B4202030B4202030B420E830A000EA
:1000A0000330A1006F200130CB206330B4206130D9
:1000B000B4202030B4206D30B4206130B4207230D0
:1000C000B4206330B4206830B4206530B420D03020
:1000D000A0000730A1006F203A286D286E28A008E4
:1000E00003197A288120A00300000000000000000E
:1000F00000006F28A108031908008120A103A003B4
:100100006F280C30A500A50B8328000000001230DA
:10011000A200A20B9028922092200000000008006C
:10012000922089280D30A400A40B94280000080018
:100130000A30A802031C08009D280630A802031CF0
:1001400008009D281030A8020001031C013EA902EE
:10015000031C0800AB280A30A8020001031C013E62
:10016000A902031C0800AB28A80086150F308605DD
:100170002808F0398604061500000611A80E0F3075
:1001800086052808F0398604061500000611C830D7
:10019000A80098200800A80086110F3086052808BE
:1001A000F0398604061500000611A80E0F308605EA
:1001B0002808F03986040615000006112830A8002A
:0801C0002330A900A220080071
:02400E00723FFF
:00000001FF
